:020000040800F2
:100000007006002095240008A5230008A7230008F7
:10001000A9230008AB230008AD230008000000005E
:10002000000000000000000000000000AF230008F6
:10003000B123000800000000B3230008B523000826
:10004000B9240008BD240008C1240008C524000804
:10005000C9240008CD240008D1240008D5240008B4
:10006000D9240008DD240008E1240008E524000864
:10007000E9240008ED240008F1240008F524000814
:10008000B9230008F9240008FD2400080125000810
:1000900005250008092500080D2500081125000880
:1000A00015250008192500081D2500082125000830
:1000B000BF23000825250008292500082D25000854
:1000C0003125000835250008392500083D250008A0
:1000D0004125000845250008492500084D25000850
:1000E0005125000855250008592500085D25000800
:1000F0006125000865250008692500086D250008B0
:100100007125000875250008792500087D2500085F
:100110008125000885250008892500088D2500080F
:100120009125000895250008992500089D250008BF
:10013000A1250008A5250008A9250008AD2500086F
:10014000B1250008B5250008B9250008BD2500081F
:10015000C1250008C5250008C9250008CD250008CF
:10016000D1250008D5250008D9250008DD2500087F
:10017000E1250008E5250008E92500080000000049
:10018000ED250008F125000838B5040001D1012053
:1001900032BD00F022F808B900F023F800F013F89F
:1001A00000F024F8FFE7416100F001F832BD20685B
:1001B000C16841F40051C16000206860202068706F
:1001C000A87000207047242068702068C16821F45E
:1001D0000051C160204600F043B904F13805687849
:1001E000704700212970204600F030BA206801696C
:1001F00021F4904101612068416921F02A01704792
:100200002DE9F843054605F138070C467878202893
:10021000164698463CD1002C14BF002E012038D041
:100220003878012834D001213970212000217960EB
:10023000787000F069FAAE848146EE8403E02968A4
:1002400014F8010B4860E88C28B3E98C481EE88458
:100250004B46A868CDF80080B0F5805F0DD100F066
:1002600024F870B920882968C0F30800486028691C
:10027000002814BF641CA41CE5E700F016F8002851
:10028000DDD0032005E0202078700020387000E0E9
:100290000220BDE8F283CDF800804B4600224021C9
:1002A00000F005F80028EED0EBE700228021284678
:1002B0008DE038B5044604F138051346A8782028A7
:1002C0003ED109B1180001D1012032BD28780128A2
:1002D00036D001222A70A162A38500206860222006
:1002E000A870626B0FF25D00D063626B0FF28D003D
:1002F0001064626B0FF28D00D0640020626B106599
:100300000A462068011D606B00F077FA002000901B
:1003100020680168009142680092002200992A70CA
:10032000C26842F48072C2602068416941F00101F4
:1003300041612068416941F040014161002032BDC6
:10034000022032BD816B00680268D30513D40020FF
:10035000C8850868C26822F48072C2600868426971
:100360005208520042610868426922F0400242612C
:10037000202081F83A00084600F069BC806B00F04C
:1003800093BC000038B5846B2068406904F13905DE
:100390002978212906D1000604D50020E0842046D2
:1003A00000F047F8206840696978222906D14006A4
:1003B00004D50020E085204600F044F8E06B40F0D2
:1003C0001000E0632046BDE8324000F06EBC2DE92D
:1003D000F041069C05460E4690461F462868016877
:1003E0003140B1420CBF01200020404517D114F12B
:1003F000010FF3D024B100F087F9C01B8442EDD285
:100400002868C16821F4D07100F00CF805F13800BB
:1004100020214170817000210170032000E0002044
:10042000BDE8F081C160286841694908490041611F
:1004300070470168CA6822F0C002CA60202180F8B3
:10044000391070470168CA6822F49072CA60016866
:100450004A69520852004A61202180F83A107047D8
:100460002DE9F0470446642521680A69E06822F412
:10047000405202430A611926CA6848480240A068EF
:1004800002432069024360690243E0690243CA6093
:100490004A69A06922F4407202434A61E369404814
:1004A000404AB3F5004F3BD1914218BF814210D171
:1004B00000F089FC074600F086FC804600F083FCD3
:1004C000814600F080FC06FB09F9824600F07BFCC7
:1004D0000FE000F070FC074600F06DFC804600F075
:1004E0006AFC814600F067FC06FB09F9824600F0D1
:1004F00062FC6168490000F057F8DB003233B3FB5F
:10050000F5F35B00B2FBF5F203F4F87300F05AF870
:10051000ED0032356420B5FBF0F000F0070037E065
:10052000914218BF81420ED100F04DFC074600F009
:100530004AFC804600F047FC814600F044FC8246BD
:1005400000F041FC0DE000F036FC074600F033FC03
:10055000804600F030FC814600F02DFC824600F021
:100560002AFC06FB09F96168890000F01DF81B01EF
:100570003233B3FBF5F3B2FBF5F203F0F00300F016
:1005800021F82D0132356420B5FBF0F000F00F00AA
:100590002168C3188B60BDE8F0870000F369FFFF96
:1005A00000140140001001407743B7FBF1F206FB55
:1005B00008F7B7FBF1F3B9FBF1F7B7FBF5F705FB6C
:1005C0001733704703EB021306FB0AF74643B7FBEA
:1005D000F1F2B6FBF1F06421B0FBF1F005FB102560
:1005E0007047000082B0002000900022404841681F
:1005F00041F480414160416801F4804100910099DB
:100600000092036843F080530360006800F080505C
:1006100000900098072002B000F027BC0068B0F1FD
:10062000804F00D0704780B50021314800910268AA
:1006300042F001020260002200F054F81C2000F099
:1006400021FCBDE802401C2000F039BC38B586B062
:10065000044601A8142100F05DFC2168254A91425E
:100660003ED10020009000222348244D016941F42E
:1006700000310161016901F400310091009900929B
:100680000C21036843F001030360022200F02AF802
:10069000019101200390032107200491059002920B
:1006A00001A9174800F03AFC164828604FF0006096
:1006B00068600020A860E8604FF480602861002036
:1006C0006861A8614FF48070E86100202862686268
:1006D000284600F01FF808B100F0D6FA6563AC6355
:1006E00007B030BD006800F001000090009870472E
:1006F000403802400044004030380240D801002019
:10070000000002408860024001484068704700BF16
:10071000400000207CB50446FFF7F6FF06460CB902
:10072000012076BD04F13405002028700220687095
:1007300000F065F921680868C20720D5FFF7E4FFDB
:10074000801B0628F6D320202862032015E0B0F590
:10075000005F09D1032E42D8DFE806F00C0A0C0234
:10076000B1F1C07F3BD105E0022E03D9F61E36D190
:10077000C80134D5402028620120687076BD0A681F
:10078000DFF86802024060680243A0680243E06844
:1007900002432069024360690243A0690243E069A1
:1007A0000243206A0243606A042803D1E36A206B93
:1007B00003431A430A6023685A69606AD20804280E
:1007C00040EAC2020BD1A66AE16A324339B1A0699C
:1007D0000028BCD1002E18BF022EC9D0C0D35A6148
:1007E000204600F027F9A96A3F228A408260002053
:1007F000286201206870002076BDF8B5044604F137
:10080000340600253078776A012801D10220F2BD34
:10081000012030707078012820D10220707035627C
:10082000204600F0F7F8B06A3F218140B9602068A7
:10083000016841F0160101602068416941F08001C2
:100840004161F06820B12068016841F00801016051
:100850002068026842F00102026001E03570022562
:100860002846F2BD2DE9FC41044604F1340600207F
:100870005F4900904FF41650776A0A683D68B2FBF2
:10088000F0F8B06A082100F0B6F80ED020680268CF
:1008900053070AD5036823F004030360B06A81405C
:1008A000B960306A40F001003062B06A25FA00F1A8
:1008B000C9070BD521684A69110607D5012101FA3C
:1008C00000F0B860306A40F002003062042100F0AD
:1008D00091F808D021680A68930704D5B860306A97
:1008E00040F004003062102100F084F81BD0216831
:1008F0000A68130717D5B860206801684A0307D54E
:10090000006801030BD5716969B1204688470AE088
:100910000168CA0503D4026822F008020260F16887
:1009200009B120468847B06A202100F064F841D020
:1009300021680A68D3063DD5B8602068717805291A
:1009400020D1026822F0160202602068416921F07D
:1009500080014161F168002904BF7069002804D05A
:100960002068016821F0080101603F22B06A8240DE
:10097000BA6000F04AF8F169002935D02046BDE898
:10098000FC41084701684A0307D5006801030DD4FC
:10099000316979B1204688470CE00168CA0505D461
:1009A000026822F01002026000F02FF8B16809B16D
:1009B00020468847306AB8B1316AC8070ED505208D
:1009C000707000F01CF820680099491C884500915F
:1009D00002D30168CA07F7D400F017F8B16919B15A
:1009E0002046BDE8FC410847BDE8F3813F8010F098
:1009F0004C000020B06A01FA00F005427047206800
:100A000001684908490001607047002030700120EA
:100A10007070704738B50468256825F48025256016
:100A200063608068402802D1A260E16031BDA160AE
:100A3000E26031BD81B0016801F0FF02103A182375
:100A4000B2FBF3F205A39B5CC365890A8902042A01
:100A500028BF091D8165084601B0704700061016C1
:100A60000006101638B586B000F05AFB00F0A5F865
:100A700001A8142100F04EFA0020794C794D009025
:100A8000216841F0010121600021206800F001008F
:100A90000090009800914FF47041226842F00802E3
:100AA00022600022206800F008000090009828468C
:100AB00000F013FB0120002101900291039101A994
:100AC000694800F02BFA4FF470400190012100209A
:100AD00002910390049001A9284600F01FFA00201B
:100AE000009000222168614D41F400112160002135
:100AF00020685F4C00F4001000900098102000F077
:100B0000C1F9102000F0DBF902A8102100F002FA70
:100B100063A0D0E900234FF08040606440F6354088
:100B2000A0640020E06401202065CDE900230020BE
:100B30006065E06504F1440000F00CFB4FF4805068
:100B4000029002A904F1440000F0D7FB00200090BD
:100B50000190694604F1440000F0C6FC454860601D
:100B60004FF4E130A0600020E060206160610C2063
:100B7000A0610020E0612062201DFFF705FB01223B
:100B80002146201DFFF795FB0A2311223FA1201DBE
:100B9000FFF736FB04F1440000F0C6FC04F144000A
:100BA00000F0E5FA201D00F099FD334C00F0C1FD86
:100BB0006868804760688047F8E780B592B006A80B
:100BC000302100F0A7F901A8142100F0A3F90020BA
:100BD00000902A48016841F08051016000210068BE
:100BE00000F0805000900098254800910221026892
:100BF00042F4804202600122006800F480400090CC
:100C00000098069110200A900C9100200D90082168
:100C100032200F900E91072004211190099210911B
:100C200006A800F077FF0F2001900221002002911A
:100C300003904FF4C0514FF4A0500491059000214F
:100C400001A800F033F813B000BD00F0C7BC08489D
:100C50000078A0F1AA0103299CBF0A4908707047D7
:100C600030380240000C02400000024038020020F0
:100C7000540100200044004040020020403802405F
:100C80000070004068020020704700005541525437
:100C900020436F6E6E65637465640D0A0A00000080
:100CA0000000000000000000704770472DE9F84385
:100CB00004000F4677D0494E306800F00F00B8426C
:100CC00002D200F072F86ED12068454D810712D52E
:100CD000400703D5A86840F4E050A86021780807D1
:100CE00003D5A86840F46040A860A968A06821F016
:100CF000F0010143A9602078C1074CD56068012844
:100D000002D129688A0305E0022818BF032803D10D
:100D100029688A0103D446E02A68910743D5A96867
:100D2000890840EA8100A86041F28939FFF7ECFCAC
:100D30008046A868616800F00C00B0EB810F2AD0F3
:100D4000FFF7E2FCA0EB08004845F2D3032020E0C7
:100D50002078410705D5A968E06821F4E0510143F6
:100D6000A9602078010706D5A868216920F46040B1
:100D700040EAC100A86000F03DF8AA681949C2F332
:100D80000312895C184AC8401060002001F03AF84C
:100D90000020BDE8F283306800F00F008742D7D210
:100DA00000F003F8D4D00120F3E73770316801F088
:100DB0000F01B94270470C480C4A006813680C498F
:100DC000C3F3822206E00848084A0068136808490D
:100DD000C3F34232895CC84070470000003C0240C7
:100DE00000380240D42200084C000020083802409D
:100DF000B024000818B5124C606800F00C000428FC
:100E000002D0082802D019E00E4812BD0023226843
:100E1000206841022068C0F388104CBF09490A4984
:100E200002F03F02A1FB000101F00CF82168C1F3C0
:100E30000141491C4900B0FBF1F012BD024812BD4E
:100E40000438024000127A000024F4000901020074
:100E500081B002D42948815405E0294802F00F02EC
:100E6000104400F8041C01B07047264A13684FF67E
:100E7000FF0100020B4000F4E060184322490843E0
:100E80001060704738B51F4B1C68C4F30223C3F1D0
:100E90000704052C28BF04241D1D072D34BF002383
:100EA000DB1E012505FA04F4641E2140994005FA71
:100EB00003F35B1E1A401143BDE83440C6E701004E
:100EC00007D4012200F01F01104B8A40400943F86B
:100ED0002020704710B5401EB0F1807F01D3012063
:100EE00010BD0B4C60600F214FF0FF30FFF7AEFFDD
:100EF0000022A26007202060002010BD00E400E076
:100F000018ED00E00CED00E00000FA0500E100E063
:100F100010E000E0002201F0ADB800002DE9F84F2C
:100F20004FF0000E734A744BDFF8D0814FF00F0979
:100F300006468A460121DAF8004001FA0EF10C401B
:100F40008C4240F0BC80DAF80450022D18BF122DFC
:100F50004FEA8E0012D14FEADE0506EB850C00F059
:100F60001C05DCF8207009FA05FB27EA0B07DAF804
:100F700010B00BFA05F53D43CCF820504FEA4E0C6B
:100F8000032537689AF804B005FA0CF5ED430BF029
:100F9000030B2F400BFA0CFB4BEA07073760DAF81C
:100FA0000470012F18BF022F03D0112F18BF122F6A
:100FB00013D1B768DAF80CB02F400BFA0CFB4BEAF0
:100FC0000707B760776827EA0101DAF80470C7F30A
:100FD000001707FA0EF739437160F1680D40DAF82F
:100FE000081001FA0CF12943F160DAF80410C90085
:100FF00065D50025009500F00C00D8F8001041F4EC
:101000008041C8F8001009FA00F7D8F8005005F43C
:101010008045009500994FEA9E0153F8215025EA3A
:101020000707374DAE4208BF002522D0354DAE42EE
:1010300008BF01251DD0344DAE4208BF022518D08F
:10104000324DAE4208BF032513D0314DAE4208BF2A
:1010500004250ED02F4DAE4208BF052509D02E4DD8
:10106000AE4208BF062504D02C4DAE420CBF07256A
:10107000082505FA00F0384343F82100E0431168E1
:10108000DAF804500140ED0348BF21431160516874
:10109000DAF804500140AD0348BF21435160916824
:1010A000DAF804500140ED0248BF21439160D16855
:1010B0000140DAF80400800248BF2143D1600EF1FC
:1010C000010EBEF10F0F7FF635AFBDE8F18F00695D
:1010D000084018BF0120C0B2704781B002B90904AE
:1010E00005E081B042690A408A4208BF0904816173
:1010F00001B07047003C01400838014044380240CC
:10110000000002400004024000080240000C0240BF
:10111000001002400014024000180240001C02406F
:1011200080B50B48016841F400710160026842F427
:1011300080620260016841F4807101600320FFF762
:1011400094FE002000F05EFEFFF74CFA002002BD86
:10115000003C024038B5040001D1012032BD00F04E
:1011600024F818B900F01DF8FFF758FA0FE00068EE
:10117000C16841F00101C160816801F007010629E1
:1011800003D0016841F00101016000207047022096
:101190006870211D206800F00DF9012068700020A2
:1011A00032BD002129702046704704F13C05687863
:1011B000704710B50446206801698A0715D5C168D3
:1011C0008A0712D56FF0020202610121217780693E
:1011D00010F0030F204602D000F065FF03E000F09E
:1011E00063FF00F087F800202077206801694A0734
:1011F00015D5C1684A0712D56FF0040202610221B9
:101200002177806910F4407F204602D000F04BFF28
:1012100003E000F049FF00F06DF80020207720681F
:1012200001690A0715D5C1680A0712D56FF00802CF
:10123000026104212177C06910F0030F204602D01B
:1012400000F031FF03E000F02FFF00F053F8002022
:10125000207720680169CA0615D5C168CA0612D56B
:101260006FF01002026108212177C06910F4407FFD
:10127000204602D000F017FF03E000F015FF00F059
:1012800039F80020207720680169CA0708D5C168AD
:10129000CA0705D56FF0010202612046FFF7D5FCB1
:1012A000206801690A0608D5C1680A0605D56FF0ED
:1012B00080020261204600F0F8FE206801694A06BB
:1012C00008D5C1684A0605D56FF040020261204684
:1012D00000F0ECFE206801698A060AD5C1688A061A
:1012E00007D56FF0200202612046BDE8104000F0F3
:1012F000DEBE10BD204600F0DBBE38B500F04FF872
:1013000001D1022032BD01222270022060702A68C1
:10131000DFF838019368034093600868020018BF43
:1013200010282DD0202818BF302829D0402823D0BD
:10133000502816D0602818D0702803D0B0F5005F70
:1013400007D021E000F026F82868816841F0770195
:1013500005E000F01FF82868816841F48041816051
:1013600012E000F013F850210BE0CA6849682868C1
:1013700000F093F8602104E000F008F8402100E05C
:101380000146286800F09BF80FE00000CA68496831
:10139000286873E0CB684A688968286897E0054642
:1013A00005F13C042078012870470120607000207E
:1013B000207032BDF0B5264C0568264B264E274FCF
:1013C000DFF89CC0A04218BFB0F1804F07D0604545
:1013D00018BFB84203D0B04218BF98420DD14A6836
:1013E00025F070051543A04218BFB0F1804F17D00B
:1013F00060451CBFB842B04212D098421CBF194A87
:1014000090420DD0184A90421CBF184A904207D013
:10141000174A90421FBF174A9042174A904203D181
:10142000CA6825F4407515434A6925F080051543BF
:101430000560A0428A68C2620A68826212BF98424E
:101440000969016301214161F0BD00008800FFFFCF
:101450000000014000040140000C00400008004072
:1014600000040040004001400044014000480140A9
:1014700000180040001C00400020004010B5036A26
:10148000046A64086400046223F00A03846924F097
:10149000F00444EA0214846123E010B5036A23F0E7
:1014A000100303628369046A23F4704343EA02333E
:1014B00024F0A004836144EA0114046210BD826830
:1014C00022F07002114341F007018160704710B5AE
:1014D000846824F47F442143114341EA032181605D
:1014E00010BD1943016210BD70B500F13C031A78BC
:1014F000012A01D1022070BD01241C7002225A7001
:1015000004686568A6684A68096825F070050D4397
:10151000656026F0800600681643866001215970D8
:101520000020187070BD000010B56A4908600020E6
:1015300000240023684A02EB0011401C10280B70A5
:101540004C708B70CB708B80CB808B600B73F1DB1E
:1015500010BD0020604A0301D15C19B1401C102865
:10156000F9DB01E00121D154C0B2704778B51128F0
:1015700004DA594D05EB00152C780CB9002072BD2A
:10158000059CE87000266E70AE80E980AC70AA60A1
:101590002B73012072BD02014F4B995C00291EBFC5
:1015A00099184A78012A01D0102801DB00207047E1
:1015B00001204870704764E0474A02EB001211783E
:1015C00000291CBF5178012901D0102801DB00201F
:1015D0007047002090800120704763E038B53D4996
:1015E0000A680068136898421ED100253A4800EB4B
:1015F00005142278012A04BF6078012811D1A0883F
:10160000E18888420BD3E078A1688847A078012858
:1016100003D1E8B200F035F803E0002000E0401C00
:10162000A0806D1C102DE1DB31BDF8B504460D46E0
:101630001646FFF78EFFFF2807460AD000960023C4
:101640002A462146FFF792FF0028384603D0FFF7CD
:10165000B3FF3846F2BD00F025F8FF20F2BD1E4B67
:1016600003EB00131A78002A1CBF5A78012A01D014
:10167000102801DB0020704700209880D9800120CD
:1016800070470201144B995C00291EBF9A185178CB
:10169000002901D0102801DB002070470020507085
:1016A000012070470C4A02EB0012117800291CBF80
:1016B0005178012901D0102801DB0020704700205B
:1016C000107050709070D0709080D0809060012029
:1016D00070470000640200205400002010B5DFF8BD
:1016E0007043206200F0E6FC40F6B83000F043FDA5
:1016F00000F072FD00F0A1FD00F0A7FD00F0ADFDCF
:1017000000F0AFFD206A0FF278310A231322FEF7B2
:1017100077FD0020207000210FF21D00606021760F
:1017200000F090F9002020740FF27D106061E061FC
:1017300010BD00F0E4BC000080B500F037FD70B9CA
:1017400000F008FD58B100F00FFD40B100F06EF858
:1017500000F069F800F02DFDDFF8F80269E001BD46
:1017600010B500F023FDB0B900F0F4FCDFF8E4425E
:1017700050B100F0F9FC38B100F058F800F053F81F
:1017800000F017FDA068804700F021F803D100F0B9
:1017900010FDE06884E010BD10B500F007FDA8B9A9
:1017A00000F0D8FCAB4C50B100F0DEFC38B100F0DA
:1017B0003DF800F038F800F0FCFC2069804700F0AC
:1017C00006F803D100F0F5FC606969E010BDA2489D
:1017D0000178AA29704710B500F0E8FCA0B900F024
:1017E000B9FC9C4C50B100F0BFFC38B100F01EF8C1
:1017F00000F019F800F0DDFCA0698047FFF7E7FF73
:1018000002D100F0D6FC4AE010BD80B500F0A2FC89
:1018100040B100F0A9FC28B100F008F800F003F88E
:101820008E4806E001BD002000F09BBC002000F0C7
:101830008EBC0168BDE80140084780B500F08AFC15
:1018400048B100F091FC30B1FFF7F0FFFFF7EBFF7C
:1018500082488168EEE701BD80B500F07BFC48B1AD
:1018600000F082FC30B1FFF7E1FFFFF7DCFF7B48BF
:101870000169DFE701BD10B500F06CFC774C40B1A9
:1018800000F072FC28B1FFF7D1FFFFF7CCFFA06991
:10189000804771480178AB2900D100E010BDE069B4
:1018A000BDE81040004700007047000038B500F068
:1018B000DCFC00F064F8FA2100F09CF858B1644DAB
:1018C00074A100F021F800F0BAFC00F055F80120F6
:1018D00028706348686031BD7047000038B500F07B
:1018E000C4FC00F04CF800F083F860B1DFF8605100
:1018F0006CA100F009F800F0A2FC00F03DF8022015
:1019000028705848686031BD286A0A230D22FEF706
:1019100077BC75E038B500F0A8FC00F030F84FF463
:101920007A7100F067F860B1DFF8245161A1FFF728
:10193000EBFF00F084FC00F01FF8032028704A48F9
:10194000686031BD5CE05BE05AE0000038B500F053
:101950008FFC00F014F8FA2100F04CF858B13C4D1F
:1019600058A100F027F800F074FC00F005F8012001
:1019700028723E48E86031BD2046FFF70CBE0446A1
:10198000FFF719BE7047000038B500F071FCFFF793
:10199000F6FF00F02DF860B1DFF8B4504DA100F073
:1019A00009F800F056FCFFF7E7FF022028723048E4
:1019B000E86031BD286A0A230E22FEF721BC31E01F
:1019C00038B500F055FCFFF7DAFF4FF47A7100F0FC
:1019D00011F860B1DFF8785042A1FFF7EBFF00F09B
:1019E00038FCFFF7C9FF032028722248E86031BDA8
:1019F0004FF4FA712046FFF732BE13E012E011E017
:101A000010B500F032FC124CFFF7D5FDD4F82000E1
:101A100038A1FFF77AFF00F010FC00202070164874
:101A2000606010BD10B500F023FC094CFFF7C3FD4A
:101A3000D4F8200033A1FFF7BEFF00F006FC00F051
:101A400001F810BD002020720C48E06070470000D3
:101A50003802002000000020680200202000002042
:101A60006117000899170008D71700083B180008ED
:101A70005918000877180008391700080B180008D3
:101A80004D6F646520312052656420537461746524
:101A90000D0A0A00526564205374617465320D0AA0
:101AA0000A000000526564205374617465330D0AA6
:101AB0000A000000526564205374617465340D0A95
:101AC0000A000000426C7565205374617465320D24
:101AD0000A0A0000426C7565205374617465330D09
:101AE0000A0A0000426C7565205374617465340DF8
:101AF0000A0A0000526564205374617465310D0A4E
:101B00000A000000426C7565205374617465310DE4
:101B10000A0A00002DE9F843040017D02078B54EDA
:101B2000C10741D5B06800F00C00042807D0B068A8
:101B300000F00C0008280BD17068410208D531680C
:101B4000880331D56068002840F0B68001204FE15D
:101B50006068B0F5803F06D0B0F5A02F316807D19E
:101B600041F480213160306840F48030306006E01C
:101B700021F480313160326822F480223260606862
:101B800068B1FEF7C1FD05463168880300F1948015
:101B9000FEF7BAFD401B6528F6D3032028E1FEF7C7
:101BA000B3FD05463068810340F18680FEF7ACFD49
:101BB000401B6528F6D3F0E7FEF7A6FD401B022880
:101BC00040F2A780E9E7E06870B101213960FEF7D3
:101BD0009BFD05463068810700F1CB80FEF794FD40
:101BE000401B0228F6D9D8E73860FEF78DFD054680
:101BF0003068810763D5FEF787FD401B0228F7D9BF
:101C0000CBE70860FEF780FD0546706F810775D54C
:101C1000FEF77AFD401B0228F7D9BEE70528306F92
:101C200006D140F004003067306F40F0010005E05D
:101C3000400840003067306F20F00400306741F208
:101C40008938A06868B1FEF75FFD8146306F810773
:101C500000F19C80FEF758FDA0EB09004045F5D34C
:101C60009BE7FEF751FD8146306F810740F18E8082
:101C7000FEF74AFDA0EB09004045F5D38DE7FEF7DE
:101C800043FD401B022840F2968086E7FEF73CFDAC
:101C9000001B022840F2A7807FE700203866FEF78D
:101CA00033FD04463068810140F1A180FEF72CFD30
:101CB000001B0228F6D970E720784F4F81071BD50B
:101CC000B06810F00C0F09D0B06800F00C000828C4
:101CD0007FF479AF706841023FF575AF31688807CE
:101CE00003D5E06801287FF431AF3168206921F025
:101CF000F80141EAC0013160217808070DD560691B
:101D00003E4900283FF47DAF01220A60FEF7FCFC4B
:101D10000546706F81077FF54FAF217848073AD5A8
:101D2000306C0025C1000AD400950125306C40F0CC
:101D300080503064306C00F0805000900098DFF8E4
:101D4000C080D8F80010C8051BD4D8F8000040F4B3
:101D50008070C8F80000FEF7D7FC8146D8F8001064
:101D6000C8050ED4FEF7D0FCA0EB09000228F5D977
:101D700013E73068216920F0F80040EAC1003060C4
:101D8000BAE7A06801287FF449AF4DE71DB1306C78
:101D900020F080503064A06948B3B16801F00C01B4
:101DA00008293FF4D3AE02287FF477AF00203866CD
:101DB000FEF7AAFC0546306881013FF560AFE16996
:101DC000206AA26A0143606A520841EA8011521EE9
:101DD000E06A41EA024141EA00617160012139662D
:101DE000FEF792FC0446306881017FF54FAF00207A
:101DF000BDE8F2830038024000004742800E4742AF
:101E00000070004038B50D4D0D4A297804464FF456
:101E10007A70B0FBF1F11068B0FBF1F0FFF75AF8FF
:101E200050B9102C08D2002221464FF0FF30FFF7A6
:101E300029F8AC60002032BD012032BD40000020F6
:101E40004C000020B3BBD9B1B2F5803F7DD2022A4D
:101E50001ED98C46B1FBF2F102FB11C31B0443EA0D
:101E60001043B3FBF2FC02FB1C3380B240EA034395
:101E7000B3FBF2F002FB103240EA0C400023704743
:101E8000022A05D98446B0FBF2F002FB10C270476B
:101E90004AB105D100F0010249085FEA30007047FD
:101EA00000220023704700F0EBB90B000200002174
:101EB00000207047904271EB030CF6D3B3F5803FDE
:101EC0002FD2F0B5B3FA83F7B1FA81F4A7F10F0E70
:101ED0003D1B5340CEF1200602FA0EF2F34153406F
:101EE000B5F10F0746D80F3C2C444140C4F1200601
:101EF000A040F1414140B1FBF3F603FB1611A2FBF8
:101F00000645001BA94102D2761E8018594180EA7D
:101F1000010221FA0EF362FA0EF200215A40304615
:101F2000F0BD30B4B1FBF3FC03FB1C11A2FB0C456C
:101F3000001BA94103D2ACF1010C8018594130BCFF
:101F400002460B46604600217047B2F1807F65D3A0
:101F5000F0B5B2FA82F7B1FA81F4C7F10F063D1B72
:101F600022FA06F307F1110EF24120355A40B5F17D
:101F70000F07B8D94140C4F12006A040F1414140CB
:101F8000B1FBF3FC03FB1C11A2FB0C45001BA94198
:101F900003D2BCF1010C801859410F2F12D30F3F0F
:101FA000C90341EA5041B1FBF3F603FB1611A2FB52
:101FB0000645D4EBC030A94102D2761E80185941A3
:101FC00046EACC3C07B34140C7F12006B840F14196
:101FD0004140B1FBF3F603FB1611A2FB0645001BC3
:101FE000A94102D2761E8018594180EA010221FAE5
:101FF0000EF3C7F1200462FA0EF20CFA07F05A4011
:102000002CFA04F13043F0BD80EA010221FA0EF30C
:10201000002162FA0EF260465A40F0BD8C46B1FBD8
:10202000F2F102FB11C31B0243EA1063B3FBF2FCA3
:1020300002FB1C331B024CEA002043EA1063B3FB93
:10204000F2FC02FB1C331B024CEA002043EA106343
:10205000B3FBF2FC02FB1C331B024CEA002043EAF8
:102060001063B3FBF2FC02FB1C324CEA002000239D
:102070007047000000B500BF130096469446103923
:1020800028BFA0E80C50FAD85FEA417C28BF0CC0FA
:1020900048BF40F8042BC90728BF20F8022B48BFCF
:1020A00000F8012B00BD70477047704770477047BC
:1020B000704700001CB5464C002020706070E07036
:1020C0002071E080FF206071FFF743FAA070A078D4
:1020D000FF2813D0012100910023A0780FF25102B4
:1020E000FA21FFF743FA0028A07803D0BDE8164094
:1020F000FFF762BABDE81640FFF76FBA13BD10B51F
:10210000334C2178002904BF607800280FD10121C9
:102110003048FEF7DCFF012809D101212170A078A9
:10212000FFF74AFAA078BDE81040FFF734BA10BDB7
:102130000121284810B5FEF7CAFF0128244C02D11E
:102140000121617010BD00206070207010BD204919
:10215000087070471E490A780020012A08BF012034
:1021600070471B494870704719494A780020012A76
:1021700008BF0120704738B5154D69790024FF2943
:102180000ED10122EA70E8800FF21901E888FFF70A
:102190004CFA68716879FF2812BF0124EC70EC805A
:1021A000204632BD0A49002008717047084800796E
:1021B000704710B5064CE07840B10121217160797B
:1021C000FFF7FAF96079FFF7E6F9012010BD00008A
:1021D0005C0200200000024010B500220FF239011D
:1021E000254C00F014F8207000220FF2350100F0A9
:1021F0000EF8607000220FF2350100F008F8A070B0
:1022000000220FF2310100F002F8E07010BD4FF42F
:102210007A70FFF70ABA00004FF4804102E0000034
:102220004FF400411548FEF75CBF00004FF48051A9
:10223000F8E700004FF40051F4E7012200E000222B
:102240004FF480410D48FEF748BF01224FF4004192
:10225000F8E700224FF40041F4E701224FF48051E7
:10226000F0E701224FF40051ECE703480078704793
:10227000014840787047000050000020000C0240E8
:10228000704700000E48016841F4700101600022AF
:102290000C49086840F0010008608A600A480A6832
:1022A00002400A60002209484860086820F4802043
:1022B0000860CA604FF00060054908607047000080
:1022C00088ED00E000380240FFFFF6FE10300024E9
:1022D00008ED00E00000000000000000010203041F
:1022E00006070809AD180008D9180008DD1800080D
:1022F00013190008151900084519000847190008A6
:10230000491900084D1900088519000889190008A5
:10231000BF190008C1190008FB190008FD190008C1
:10232000FF1900080100000000000000100000007C
:102330000024F400FFFFFFFF19E050F8042BD3073F
:1023400044BFA9F101039A18091F0023042942F888
:10235000043BF9D25FEA817C134604D54FF0000CB0
:10236000A2F800C09B1CC90744BF0021197050F897
:10237000041B0029E1D1704710B450F8041B79B157
:102380000268436802440830DC0744BFA9F1010435
:10239000E31852F8044B43F8044B091FF9D1ECE75A
:1023A00010BC70477047FEE7FEE7FEE7FEE77047A8
:1023B0007047704700F00AB80248FEF753BA024867
:1023C000FEF7F7BED80100209801002002484168BE
:1023D00002788918416070474000002010B5074915
:1023E00079441831064C7C44163404E00A68081D10
:1023F000114488470146A142F8D110BD2C000000CD
:102400004C0000004EF68851CEF20001086840F4FE
:1024100070000860BFF34F8FBFF36F8F4FF00070F5
:10242000E1EE100A7047000011FFFFFF18020000E4
:10243000540000200000000041FFFFFF5400000096
:10244000A4FEFFFF000000200000000000F00DF8D7
:10245000002801D0FFF7C2FFAFF300800020AFF3E8
:102460000080FEF7FFFA00F002F80120704700F04C
:1024700001B800000746384600F002F8FBE700000C
:1024800080B5AFF30080024A11001820ABBEFBE715
:1024900026000200014880470148004785220008C5
:1024A000A5240008AFF30080FFF7ACFFFFF7CEFFD5
:1024B0000000000001020304FFF7FEBFFFF7FEBFAC
:1024C000FFF7FEBFFFF7FEBFFFF7FEBFFFF7FEBF40
:1024D000FFF7FEBFFFF7FEBFFFF7FEBFFFF7FEBF30
:1024E000FFF7FEBFFFF7FEBFFFF7FEBFFFF7FEBF20
:1024F000FFF7FEBFFFF7FEBFFFF7FEBFFFF7FEBF10
:10250000FFF7FEBFFFF7FEBFFFF7FEBFFFF7FEBFFF
:10251000FFF7FEBFFFF7FEBFFFF7FEBFFFF7FEBFEF
:10252000FFF7FEBFFFF7FEBFFFF7FEBFFFF7FEBFDF
:10253000FFF7FEBFFFF7FEBFFFF7FEBFFFF7FEBFCF
:10254000FFF7FEBFFFF7FEBFFFF7FEBFFFF7FEBFBF
:10255000FFF7FEBFFFF7FEBFFFF7FEBFFFF7FEBFAF
:10256000FFF7FEBFFFF7FEBFFFF7FEBFFFF7FEBF9F
:10257000FFF7FEBFFFF7FEBFFFF7FEBFFFF7FEBF8F
:10258000FFF7FEBFFFF7FEBFFFF7FEBFFFF7FEBF7F
:10259000FFF7FEBFFFF7FEBFFFF7FEBFFFF7FEBF6F
:1025A000FFF7FEBFFFF7FEBFFFF7FEBFFFF7FEBF5F
:1025B000FFF7FEBFFFF7FEBFFFF7FEBFFFF7FEBF4F
:1025C000FFF7FEBFFFF7FEBFFFF7FEBFFFF7FEBF3F
:1025D000FFF7FEBFFFF7FEBFFFF7FEBFFFF7FEBF2F
:1025E000FFF7FEBFFFF7FEBFFFF7FEBFFFF7FEBF1F
:0425F000FFF7FEBF34
:04000005080024A526
:00000001FF
